:0300000002303596
:0C30350078FFE4F6D8FD75814A02307C7B
:100DF2000A53746172743A20004950436F6E6E65F3
:100E020063745245510A004950436F6E6E656374B4
:100E1200003E432C562C52432CC0E4E0EFF2E5F0A6
:100E220020D1E8EDEAEEEC49500A003E432C4D4158
:100E3200432C25303262583A25303262583A2530F6
:100E42003262583A25303262583A25303262583A84
:100E520025303262582C4D414320E0E4F0E5F10A9E
:100E6200003E432C5645522C20332E3120EEF220E8
:100E720025732025732CC2E5F0F1E8FF20495020AC
:100E8200ECEEE4F3EBFF0A004E6F762030332032B3
:100E92003030370030383A35323A3130003E432C68
:100EA2004C442C50524F473A202020202020202012
:100EB2002020202020202020202020202020202030
:100EC2002020202020202020202020202020202020
:100ED2002020202020202020202020202020202010
:100EE200202020202020202020202020202CC4E090
:100EF200F2E020EFF0EEF8E8E2EAE828F4E0E9EBCD
:100F0200290A003E2A2C312CCEF1EDEEE2EDFBE572
:100F120020EFE0F0E0ECE5F2F0FB20F1E5F2E5E2B3
:100F2200EEE3EE20E8EDF2E5F0F4E5E9F1E00A00A7
:100F32003E412C4130312C2562752E2562752E25BD
:100F420062752E2562752C495020E0E4F0E5F1200F
:100F5200E0E4E0EFF2E5F0E00A003E412C413032FD
:100F62002C2562752E2562752E2562752E256275D9
:100F72002C495020E0E4F0E5F120EEF1ED2E20F1D5
:100F8200E5F0E2E5F0E00A003E412C4130332C2549
:100F920062752E2562752E2562752E2562752C4985
:100FA2005020E0E4F0E5F120F0E5E72E20F1E5F055
:100FB200E2E5F0E00A003E412C4130342C25627516
:100FC2002E2562752E2562752E2562752CCCE0F1D8
:100FD200EAE020F1E5F2E80A003E412C4130352CEE
:100FE2002562752E2562752E2562752E2562752C59
:100FF200D8EBFEE70A003E532C4130362C256275B1
:101002002CC2F0E5ECFF20EEE6E8E42E20EAE2E86E
:10101200F2E0EDF6E8E820282A3130ECF1290A0066
:101022003E2A2C312CC4EEEF2E20EFE0F0E0ECE56E
:10103200F2F0FB20F1E5F2E5E2EEE3EE20E8EDF27C
:10104200E5F0F4E5E9F1E00A003E422C5330312CA0
:101052002562752CC6E4E0F2FC20E7E0EFF0EEF149
:10106200E020F1EEE5E4E8EDE5EDE8FF20EEF22028
:10107200F1E5F0E2E5F0E00A003E422C5330322C7A
:101082002562752CCEE1ECE5ED20F120F1E5F0E2F0
:10109200E5F0EEEC20E1E5E720EAE2E8F2E0EDF649
:1010A200E8E90A003E422C5330332C2562752CCFDE
:1010B200E5F0E5E7E0EFF3F1EA20EFF0E820EFEE0C
:1010C200F2E5F0E520F1E2FFE7E820F120F1E5F0BA
:1010D200E2E5F0EEEC0A003E422C5330342C25625D
:1010E200752CCDE5F220EFE5F0E5E4E0F7E820E449
:1010F200E8E0E3EDEEF1F2E8EAE820E220F1E5F0E3
:10110200E2E5F00A003E422C5330352C2562752C64
:10111200CAE0EDE0EB20F8E8F0EEEAEEE2E5F8E016
:10112200F2E5EBFCEDEEE3EE20EEE1ECE5EDE00ABC
:10113200003E532C5330362C253032625825303243
:101142006258253032625825303262582530326278
:101152005825303262582C4D414320E0E4F0E5F14D
:1011620020F8E8F0EEEAEEE2E5F8E0F2E5EBFCED7D
:10117200EEE3EE20EEE1ECE5EDE00A003E454E4402
:101182000A0044756D705820202020203030203015
:101192003120303220303320303420303520303688
:1011A2002030372030382030392030412030422062
:1011B20030432030442030452030460A003A200097
:1011C2000A0044756D7044202020202030302030E9
:1011D2003120303220303320303420303520303648
:1011E2002030372030382030392030412030422022
:1011F20030432030442030452030460A0045727288
:10120200206B657900526420656570726F6D0A000B
:101212005264204D454D0A00526420436F64650AB2
:101222000044656275674950204F4E0A004465626A
:1012320075674950204F46460A00446562756755F6
:10124200736572204F6E0A00446562756755736557
:1012520072204F46460A0044656275674D736720E7
:101262004F6E0A0044656275674D7367204F4646AC
:101272000A00436F6E666967206C6F636B210A0018
:10128200577220656570726F6D0A00205361766532
:1012920020656570726F6D210A00457272204D41A2
:1012A2004321004C6F61643E3E002A003C413031D4
:1012B2003D003C4130323D003C4130333D003C4139
:1012C20030343D003C4130353D003C4130363D003C
:1012D2004E4F4950004C494E4B434F4E54520054CE
:1012E20052415353004652004E4F4C494E4B004917
:1012F2004E49004E4F4449414700003C21003C53B7
:1013020030313D003C5330323D003C5330333D00E0
:101312003C5330343D003C5330353D003C53303675
:101322003D00FF12D2FF12D7FF12E1FF12E7FF12B8
:0A133200EAFF12F1FF12F5FF12FCB2
:06385800014700014500DC
:10388E00C2AFC28E438910758BFF758DB7D2ABD286
:04389E008ED2AF22F5
:03001B00022E644E
:102E6400C0E0C083C082C0D0C2AFC28E758BFF7574
:102E74008DB720160675A61E75A6E10545D212E586
:102E84004760020547E546D3940140021546054ACA
:102E9400E54A540F7050D21DE54A543F701AD210BF
:102EA40090668DE0601204F0E0D394B4400A908000
:102EB400007480F0C2AF80FE906688E0600204F087
:102EC400906104E0600214F090668EE0D3940140B7
:102ED40003E014F03015020548E549D39464400436
:102EE400D21680020549E544D3940140021544D228
:0C2EF4008ED2AFD0D0D082D083D0E0329C
:10087D00C21A7D027C007F0712383B8F25E5256467
:10088D006060097D017F601237D3D21AE4FDFC7FD1
:10089D000B12383B8F25E52530E6097D04E4FF1268
:1008AD0037F7D21A7D017C007F0712383B8F25E583
:1008BD00257008FD7FFF1237D3D21A301A0312604C
:1008CD0000C2AFC288C2A8C2AA758900122F00D279
:1008DD00AF90634C7403F0A374CCF0E490634BF0D1
:1008ED00122845EF6003121E1C123439C216123540
:1008FD00D6906358E0C3940350037403F0D21AC228
:10090D001CC21BD293201A077E0D7FF212292BE4F5
:10091D00906578F012388EC2AFA37408F09062B76C
:10092D007424F0E4A3F0906341E09062B9F0906319
:10093D0042E09062BAF0906343E09062BBF0906346
:10094D0044E09062BCF0906345E09062BDF090632E
:10095D0046E09062BEF0754601E490657AF0C217EC
:10096D00C218D2AF75A70775A61E75A6E1201A1875
:10097D00AF25FE7D03122A0CE4FF122C6F7E637FE0
:10098D0078E4FB7D01122AE690668DE06003740128
:10099D00F0E4906104F0A37455F0A37481F0E4F5D4
:1009AD0048E4F549906104E0700312372490668E97
:1009BD00E0B401119080007410F0E490668EF0D2D6
:1009CD001AD21BD21C908008E0F52530E405D21711
:1009DD007410F0E52530E508D2199080087420F0E8
:1009ED00E52530E608D2189080087440F0E548D32C
:1009FD0094034023908002E4F0908001F0908000F9
:100A0D00F0E548D39406400FE4F548C21390657A9B
:100A1D00F07546011235D69080A0E0700312334573
:100A2D009080B8E070031233BF9080D0E070031255
:100A3D003516908000E07013301710122640906329
:100A4D0034EFF0D394004003120026908002E07042
:100A5D0006908000E06005D2150209AEC215E4F5DE
:100A6D0048906104E060030209AE3019121224DAD5
:100A7D00906334EFF0D394004005E0FF1200222084
:100A8D001803020C08122365906334EFF070030213
:100A9D0009AE906378E054BF247F7003020B6B1492
:100AAD007003020B4324026003020B9E201A077E83
:100ABD000D7FFB12292B301E74201371906350E0B3
:100ACD00FF7006906354E06055906684E0FEB507B4
:100ADD0022A3E0FF906351E0B50718906686E0FF12
:100AED00906352E0B5070C906687E0FF906353E08A
:100AFD006F602B906354E06E7033906685E0FF90CD
:100B0D006355E0B50727906686E0FF906356E0B524
:100B1D00071B906687E0FF906357E0B5070F906560
:100B2D007A7401F012001E754601020C089066845D
:100B3D0074FFF0020C0890668DE060037401F09074
:100B4D00667CE0FF90637AE06F6003020C089066AC
:100B5D007CE004F0E4F546906578F0020C08301363
:100B6D0003020C08906347E070030209AE1238EDE2
:100B7D00D213E4F546906578F090668804F0E49021
:100B8D00667BF0A3F0201A737E0E7F0912292B804D
:100B9D006A90668DE060037401F0301352906378B3
:100BAD00E020E74B90637AE0FF90667BE0FE6F609C
:100BBD000D906683E07007EE146F703F80139066A2
:100BCD007BE004F0906334E0FFD3940440031234CF
:100BDD00B29060007482F0A37401F090637AE0909B
:100BED006002F07E607F007D031232CA0209AE30D2
:100BFD001E0920130690668474FFF0201303020C67
:100C0D00BDE546706B122F9CEF60207E647F78905F
:100C1D006479E02404FD1232CA906683E060030219
:100C2D0009AE906358E0F5460209AE906688E0D3B0
:100C3D00943C403C906683E0703690668804F0905A
:100C4D0062B6E0702B122BBAE4906478F0A37412A4
:100C5D00F090667CE090647AF0A374FDF0906107EB
:100C6D0063A20190647C63A2017F121220EA809B33
:100C7D001238D8EF60159060007483F0E4A3F07E15
:100C8D00607F007D021232CA0209AEE54664016042
:100C9D00030209AE906578E004F0E0C394055003BB
:100CAD00020C18C213E490657AF012001E0209AE10
:100CBD00E546640160030209AE90657AE014604078
:100CCD0024FE603C147003020DA524046003020988
:100CDD00AEE4F548201E1390657A7404F0906578A3
:100CED00E05401F07546010209AEE490657AF0908A
:100CFD00657804F07546C890668474FFF00209AEFD
:100D0D00906684E07003020D949064787480F09086
:100D1D00647A7401F0E4A3F0A304F0A37430F0A39B
:100D2D00747BF0E4F525747F2525F582E43464F5B4
:100D3D0083747DF074802525F582E43464F583E4B5
:100D4D00F0E5252407906479F07C667D8490634CF2
:100D5D00E0FAA3E0FB7F021231467E647F78E52541
:100D6D002409FD1232CA906683E0601B1238EDD261
:100D7D0013E4F546906578F090668804F0E490668B
:100D8D007BF0A3F00209AE90657A7404F09063587D
:100D9D00E02432F5460209AE9080027410F07546DB
:100DAD0003906578E06401FFF090657A7401F0EFCF
:100DBD007019906354E06013FCA3E0FDA3E0FEA363
:100DCD00E0FF906684121A860209AE906350E0FC33
:100DDD00A3E0FDA3E0FEA3E0FF906684121A860255
:040DED0009AE80FECD
:010DF10022DF
:10002600906379E0B444047F0180027F0090637896
:10003600E0B447047E0180027E00EE5F604A906372
:1000460041E090637AF0906342E090637BF09063C6
:1000560043E090637CF0906344E090637DF09063AE
:1000660045E090637EF0906346E090637FF0906396
:10007600797452F09062B063A2019080A863A201E5
:100086007F061220EA020873906334E0C394085096
:100096000302087C906341E0FF90637AE06F60039F
:1000A60002087C906342E0FF90637BE06F6003028E
:1000B600087C906343E0FF90637CE06F6003020876
:1000C6007C906344E0FF90637DE06F600302087CF0
:1000D600906345E0FF90637EE06F600302087C90CA
:1000E6006346E0FF90637FE06F600302087C9063E5
:1000F60079E0B444159062B0E0B4FF0E63A20190BB
:1001060080A863A2017F061220EA90668DE0600354
:100116007401F090668E7464F09063797452F09076
:100126006378E0646D60030202A37BFF7A0E7913A5
:1001360012139E7BFF7A0E792D906341E0F52EA374
:10014600E0F52FA3E0F530A3E0F531A3E0F532A307
:10015600E0F53312139E752EFF752F0E75308A75D6
:1001660031FF75320E7533967BFF7A0E7963121363
:100176009E7BFF7A0E799F12139E7BFF7A0F79057D
:1001860012139E7BFF7A0F7932906347E0F52EA318
:10019600E0F52FA3E0F530A3E0F53112139E7BFFC7
:1001A6007A0F795C906350E0F52EA3E0F52FA3E07B
:1001B600F530A3E0F53112139E7BFF7A0F798A9012
:1001C6006354E0F52EA3E0F52FA3E0F530A3E0F5A8
:1001D6003112139E7BFF7A0F79B890633DE0F52EBE
:1001E600A3E0F52FA3E0F530A3E0F53112139E7BD3
:1001F600FF7A0F79DB906339E0F52EA3E0F52FA3A4
:10020600E0F530A3E0F53112139E7BFF7A0F79F803
:10021600906358E0F52E12139E7BFF7A1079221216
:10022600139E7BFF7A10794BA21EE433F52E121330
:100236009E7BFF7A10797B906683E0F52E12139EE3
:100246007BFF7A1079A690668DE0F52E12139E7BC1
:10025600FF7A1079D99062B6E0F52E12139E7BFFD5
:100266007A117907A211E433F52E12139E7BFF7AD9
:1002760011793390667DE0F52EA3E0F52FA3E0F526
:1002860030A3E0F531A3E0F532A3E0F53312139E77
:10029600122D197BFF7A11797E12139E22906378B4
:1002A600E0644C70527E117F8412292B906380E0AB
:1002B600F526A3E0F527E4F5287D03AF27AE261241
:1002C6002A0C7E117FBF12292BAE26AF27E4FB7DB9
:1002D60010122AE67E117FC212292B74102527F5EB
:1002E60027E43526F5260528E528C3941040CA7E5E
:1002F600117FC212292B22906378E0646C705CF542
:100306002A7E117FC412292BE4F529AF2A7E007DAF
:1003160003122A0C7E117FBF12292BE4F528A82A86
:10032600E6FF74822528F582E43463F583EFF00551
:100336002A0528E528B410E67E637F82E4FB7D105B
:10034600122AE67E117FC212292B0529E529C394BC
:100356000840B87E117FC212292B22906378E06490
:100366004B7061F528746A2528F582E43463F583B9
:10037600E06032746A2528F582E43463F583E0F49C
:100386006023746A2528F582E43463F583E0FF74FC
:10039600802528F582E43463F583E0B50710052847
:1003A600E528B408C09061047432F00208739063C3
:1003B600787421F0301A030208737E117FFF122928
:1003C6002B020873906378E0B4521A201A077E1243
:1003D6007F0712292B9063787472F07E637F787D95
:1003E600081231CA22906378E064497045201A07E2
:1003F6007E127F1212292B906380E0F526A3E0F58A
:1004060027E4F528852782852683E0FF7482252840
:10041600F582E43463F583EFF00527E527700205DE
:10042600260528E528B480DC7E637F787D8A123134
:10043600CA22906378E064437079A3E06452704600
:10044600201A077E127F1A12292B906380E0F52668
:10045600A3E0F527E4F528852782852683E493FF24
:1004660074822528F582E43463F583EFF00527E5E9
:1004760027700205260528E528B480DB7E637F7891
:100486007D8A1231CA22906379E0645760030208BC
:100496007C906380E0F526A3E0F52774822528F595
:1004A60082E43463AD82FC7B80AF27AE261236F041
:1004B600020873906378E06444600302054A90631F
:1004C60080E0FF64447003020873EFB4310CC21A73
:1004D6007E127F2312292B020873906380E0B430CA
:1004E6000CD21A7E127F2F12292B0208739063807A
:1004F600E0B4320CD21B7E127F3C12292B02087309
:10050600906380E0B4330CC21B7E127F4A12292B03
:10051600020873906380E0B4340CD21C7E127F59BB
:1005260012292B020873906380E0B4350CC21C7E3E
:10053600127F6612292B020873906380E0FF120077
:1005460021020873906104E07013201A077E127F5F
:100556007412292B9063787421F002087390610459
:100566007432F0906378E0FFB4510A908000748092
:10057600F0C2AF80FEEF64577045201A077E127FE7
:100586008212292B906381E0906334F0E4F5289081
:100596006334E0FFE528C39F400302087374822595
:1005A60028F582E43463F583E0FF906380E0252834
:1005B60024AFF582E43461F583EFF0052880D0900E
:1005C6006378E064536003020678201A077E127F80
:1005D6008D12292B906341E0FF9061B8E06F703C6B
:1005E600906342E0FF9061B9E06F7030906343E042
:1005F600FF9061BAE0B50724906344E0FF9061BBC9
:10060600E0B50718906345E0FF9061BCE0B5070CC4
:10061600906346E0FF9061BDE06F6016906378746A
:1006260021F0301A030208737E127F9C12292B02D6
:100636000873E4F528E4F54974AF2528F582E43417
:1006460061F583E0FDAF281237800528E528C394BD
:10065600FE40E29080007480F0C2AFE4907FF0F03C
:10066600A3F0907FFD74AAF0A374FFF0A37455F075
:1006760080FE906378E0644F704C906380E0F526CE
:10068600A3E0F527E5274526700A201A077E127F84
:10069600A512292B201A077E127FAC12292BE4F50E
:1006A6002874822528F582E43463F583E085278261
:1006B600852683F00527E527700205260528E52807
:1006C600B480DE020873906378E0FFB4452790801B
:1006D600007480F0906380E0FDA3E0907FF0CDF0A1
:1006E600A3EDF0C2AF907FFD74AAF0A374FFF0A350
:1006F6007455F080FEEF64656003020873906380B2
:10070600E0FFA3E0907FF0CFF0A3EFF0E4F526F54D
:1007160027D3907FF1E09527907FF0E09526402142
:10072600E4F5492527FFE5263478FE7B80AD27AC26
:10073600261236F074802527F527E43526F526801F
:10074600D07E127FAE1230C1EF4E602012000390B1
:100756006347EFF0120003906348EFF01200039036
:100766006349EFF012000390634AEFF07E127FB404
:100776001230C1EF4E6020120003906350EFF0126A
:100786000003906351EFF0120003906352EFF012F2
:100796000003906353EFF07E127FBA1230C1EF4E22
:1007A6006020120003906354EFF01200039063552B
:1007B600EFF0120003906356EFF0120003906357B8
:1007C600EFF07E127FC01230C1EF4E6020120003A0
:1007D60090633DEFF012000390633EEFF0120003CA
:1007E60090633FEFF0120003906340EFF07E127FBC
:1007F600C61230C1EF4E6020120003906339EFF04D
:1008060012000390633AEFF012000390633BEFF09F
:1008160012000390633CEFF07E127FCC1230C1EFE2
:100826004E6008123579906358EFF0E4F528E4F548
:1008360049E52804FF74392528F582E43463F583F5
:10084600E0FD1237800528E528C3944340E09080F8
:10085600007480F0C2AFE4907FF0F0A3F0907FFDCB
:1008660074AAF0A374FFF0A37455F080FE7E637F34
:06087600787D081231CA72
:01087C002259
:1036B800AE07EEC39430400BEED394395005EE2498
:1036C800D0FF22EEC39461400BEED394665005EE12
:1036D80024A9FF22EEC39441400BEED39446500533
:0836E800EE24C9FF22AF062207
:103874009062AFE004F070069062AEE004F09062F3
:0A388400AEE0FEA3E0FF123676224C
:100003001238741236B8EFC454F0FEC006123874B6
:080013001236B8D0E02FFF22E5
:10357900E49068AFF01238749068B0EFF0C39430FB
:103589004018E0FFD3943950119068AFE02407F553
:1035990082E43461F583EFF080119068AFE024078D
:1035A900F582E43461F583E4F0800C9068AFE004BF
:1035B900F0E0D3940840BE752E00752F00753000D9
:0C35C900E4F5317B017A6179071221C121
:0135D50022D3
:0430C1008E2B8F2C97
:1030C5009062AEE4F0A374FFF0123874EF606EF412
:1030D500606B852C82852B83E493B507EC752D01F8
:1030E500E52C252DF582E4352BF583E493602590B9
:1030F50062AFE0252DFF9062AEE03400FE12367619
:10310500E52C252DF582E4352BF583E493B50704ED
:10311500052D80CCE52C252DF582E4352BF583E4B2
:103125009370A6E52D24FFFFE434FFFE9062AFE027
:103135002FF09062AEE03EF07E007F0122E4FEFFBC
:013145002267
:102845007E127FFD1230C1EF4E70037F01227E1391
:102855007F001230C1EF4E600C123874EF24D02483
:10286500FF921E8002D21E7E137F061230C1EF4EEC
:10287500600C123874EF24D0906683F08005E490E4
:102885006683F07E137F0C1230C1EF4E600C123858
:1028950074EF24D090668DF08005E490668DF07E0F
:1028A500137F121230C1EF4E600C123874EF24D032
:1028B5009062B6F08005E49062B6F07E137F181240
:1028C50030C1EF4E600C123874EF24D024FF921102
:1028D5008002C21190634163A20190667D63A201EB
:1028E5007F061220EA30113B7E137F1E1230C1EFA6
:1028F5004E603012000390667DEFF0120003906683
:102905007EEFF012000390667FEFF01200039066F1
:1029150080EFF0120003906681EFF01200039066DD
:0629250082EFF07F0022AA
:101E1C00C211E490668DF0D21EC214906683F090CD
:101E2C0062B6F090634163A20190667D63A2017F6C
:101E3C00061220EAE4F526E52675F003A42424F521
:101E4C0082E43413F583E493FB740193FA740293E4
:101E5C00F9121953700302200EE4F527F528FD74CE
:101E6C002F2DF582E43461F583E0FF700302200925
:101E7C00E52675F003A42424F582E43413F583E4F9
:101E8C0093FB740193FA740293F98527827583008E
:101E9C0012196CFEEFB506087528010527022005FE
:101EAC00E5287003022005EE6003022000E52624DD
:101EBC00FE6028147003021FE8147003021FEC1458
:101ECC007003021FF4147003021FF8240560030250
:101EDC00200990668D7401F0022009D211742F2D07
:101EEC00F582E43461F583E0FF642D700302200970
:101EFC001236B8EFC454F0FC74302DF582E4346122
:101F0C00F583E0FF1236B8EF2C90667DF074312D1E
:101F1C00F582E43461F583E0FF1236B8EFC454F077
:101F2C00FC74322DF582E43461F583E0FF1236B88F
:101F3C00EF2C90667EF074332DF582E43461F583DA
:101F4C00E0FF1236B8EFC454F0FC74342DF582E483
:101F5C003461F583E0FF1236B8EF2C90667FF07495
:101F6C00352DF582E43461F583E0FF1236B8EFC409
:101F7C0054F0FC74362DF582E43461F583E0FF12E5
:101F8C0036B8EF2C906680F074372DF582E434610E
:101F9C00F583E0FF1236B8EFC454F0FC74382DF51D
:101FAC0082E43461F583E0FF1236B8EF2C90668141
:101FBC00F074392DF582E43461F583E0FF1236B804
:101FCC00EFC454F0FC743A2DF582E43461F583E0EF
:101FDC00FF1236B8EF2C906682F08021D214801D4F
:101FEC009066837401F08015C21E80119062B674E5
:101FFC0001F08009E4F528F5270D021E6B05260279
:02200C001E4371
:01200E0022AF
:10362F00906579E0C3947C503D906579E0FE04F09D
:10363F0074B72EF582E43462F583EFF0BF0A27905A
:10364F006579E0FF04F074B72FF582E43462F583F7
:10365F00E4F0906579E0FF12324C9065797408F0D0
:07366F009062B8E004F022B4
:1035D6009080007480F090633963A201F583F582D0
:1035E60063A2017F081220EA90634163A2019080E2
:1035F6008863A2017F0A1220EA908092E4F0A37405
:1036060032F0A37401F090634BE0FF9080B1F0902C
:1036160080E1EFF09080957455F0A3F090800074EF
:0936260001F09080097470F0229B
:10334500908009E04410F09080A0E0706C9080A11E
:103355007482F09080A874FFF0A3F0A3F0A3F07F2F
:10336500039080AEEFF07FCBA3EFF07F039080ACAE
:10337500EFF0A374CBF09080007402F09068A31274
:103385001A92000000009068A3E0908040F09068D9
:10339500A4E0908041F09068A5E0908042F09068AC
:1033A500A6E0908043F0A3E4F0A3F0A3F0A3F0908F
:0933B5008018F0A3F0A3F0A3F0CE
:0133BE0022EC
:10351600908009E04440F09080D17482F090634C32
:10352600E0FF9080DEF090634DE0FF9080DFF0904A
:1035360080027402F09068A7121A920000000090B0
:1035460068A7E0908058F09068A8E0908059F090C5
:1035560068A9E090805AF09068AAE090805BF0A39A
:10356600E4F0A3F0A3F0A3F0908030F0A3F0A3F072
:02357600A3F0C0
:013578002230
:1033BF00908009E04420F09080B8E0706C9080B964
:1033CF007482F07F039080C6EFF07FCDA3EFF07F84
:1033DF00039080C4EFF0A374CDF09080C074FFF021
:1033EF00A3F0A3F0A3F09080017402F09068AB12E9
:1033FF001A92000000009068A7E090804CF090684F
:10340F00A8E090804DF09068A9E090804EF0906811
:10341F00AAE090804FF0A3E4F0A3F0A3F0A3F09004
:09342F008024F0A3F0A3F0A3F047
:013438002271
:103146008C268D27A907EAFDE975F018A424ACFFA3
:10315600E5F034808F82F583EDF0EBFDE975F0182C
:10316600A4FFAEF024ACFBEE34808B82F583A3ED96
:10317600F08527828C83E0FDEF24A8FFEE3480FEE5
:103186008F82F583EDF08527828C83A3E08F828E74
:1031960083A3F0852782852683A3A3E0FDE975F046
:1031A60018A424A8FFE5F03480FE8F82F583A3A33C
:1031B600EDF08527828C83A3A3A3E08F828E83A361
:0431C600A3A3F022AD
:0631CA008D2BAB07AA06E5
:1031D0009068A3E0FCA3E0FDA3E0FEA3E0F52F8E42
:1031E0002E8D2D8C2CAE02AF038E838F8263A201B5
:1031F000E52E540744C0F583852F8263A201AF2BCF
:10320000122153908000E020E5F9E4FCFDFEE52F5B
:10321000252BF52FEE352EF52EED352DF52DEC3534
:103220002CF52C908040E52CF0A3E52DF0A3E52EA5
:10323000F0A3E52FF09080007420F0AF2FAE2EADFC
:0B3240002DAC2C9068A3121A86AF2B57
:01324B002260
:0632CA008D26AB07AA06E9
:1032D0009068A7E0FCA3E0FDA3E0FEA3E0F52A8E42
:1032E000298D288C27AE02AF038E838F8263A201C3
:1032F000E529540744D0F583852A8263A201AF26CD
:10330000122153E4FCFDFEE52A2526F52AEE352997
:10331000F529ED3528F528EC3527F527908058E577
:1033200027F0A3E528F0A3E529F0A3E52AF0908093
:10333000027420F0AF2AAE29AD28AC279068A712FE
:043340001A86AF2614
:013344002266
:022C6F008F26AE
:102C7100908001E030E5037F00229068ABE0FCA387
:102C8100E0FDA3E0FEA3E0F52A8E298D288C279094
:102C9100667D63A201E529540744C8F583852A822C
:102CA10063A2017F06122169E52A2406F52AE4358B
:102CB10029F529E43528F528E43527F52790657BA2
:102CC10063A201E529540744C8F583852A8263A2DA
:102CD10001AF26122169E4FCFDFEE52A2526F52A2D
:102CE100EE3529F529ED3528F528EC3527F527901E
:102CF100804CE527F0A3E528F0A3E529F0A3E52A18
:102D0100F09080017420F0AF2AAE29AD28AC279055
:072D110068AB121A86AF2621
:012D18002298
:102640009081E0E0F52605260526052605260526C7
:1026500005260526052605260526908010E0F52985
:10266000A3E0F52AA3E0F52BA3E0F52C9081E1E0AF
:10267000F526052605260526052605260526052612
:10268000052605260526908014E0F52DA3E0F52EFD
:10269000A3E0F52FA3E0F530E52FB52B08E530B525
:1026A0002C037F0022E4F526E52F540744E0F58350
:1026B00085308263A20190637863A2017F081221B2
:1026C0008190637A63A2019062B063A2017F0612D7
:1026D00020EA906378E0F527A3E0F528E4F526905A
:1026E0006378E0702AA3E024F8F526E52F54074428
:1026F000E0F58385308274082582F582E43583F520
:102700008363A20190637863A201AF26122181AE98
:1027100027E4FCFDE5302528F530E52F3EF52FEDCB
:10272000352EF52EEC352DF52D908014E52DF0A3EA
:10273000E52EF0A3E52FF0A3E530F0908000744083
:03274000F0AF26D1
:012743002273
:102365009081E6E0F526052605260526052605269F
:1023750005260526052605260526908028E0F5294B
:10238500A3E0F52AA3E0F52BA3E0F52C9081E7E087
:10239500F5260526052605260526052605260526F0
:1023A50005260526052690802CE0F52DA3E0F52EC3
:1023B500A3E0F52FA3E0F530E4F526E52FB52B0ACC
:1023C500E530B52C05C2180224BFE52F540744F0AB
:1023D500F58385308263A20190637863A2017F084B
:1023E500122181906378E0F527A3E0F528E52845DB
:1023F5002770099080027410F07F0022906684E0B7
:10240500FFF4602D90637AE06F7076906685E0FF4B
:1024150090637BE06F706A906686E0FF90637CE076
:102425006F705E906687E0FF90637DE06F6022804D
:102435005090637AE0906684F090637BE0906685C7
:10244500F090637CE0906686F090637DE09066870F
:10245500F0906378E0702AA3E024F8F526E52F5480
:102465000744F0F58385308274082582F582E435CA
:1024750083F58363A20190637863A201AF261221DD
:1024850081AE27E4FCFDE5302528F530E52F3EF546
:102495002FED352EF52EEC352DF52DAF2CAE2BADC4
:1024A5002AAC29AB30AA2FA92EA82DD3121A754014
:1024B500099080027410F07F002290802CE52DF0A9
:1024C500A3E52EF0A3E52FF0A3E530F0908002748C
:0424D50040F0AF26FE
:0124D90022E0
:1024DA009081E3E0F526052605260526052605262C
:1024EA000526052605260526052690801CE0F529E1
:1024FA00A3E0F52AA3E0F52BA3E0F52C9081E4E014
:10250A00F526052605260526052605260526052679
:10251A00052605260526908020E0F52DA3E0F52E58
:10252A00A3E0F52FA3E0F530E4F526E52FB52B0A55
:10253A00E530B52C05C219022625E52F540744E8D3
:10254A00F58385308263A20190600463A2017F0E45
:10255A00122197906004E0F527A3E0F52890600C1B
:10256A00E0FFF4604590667DE0FEEF6E706EA3E0DA
:10257A00FF90600DE06F706490667FE0FF90600EE0
:10258A00E06F7058906680E0FF90600FE06F704CCB
:10259A00906681E0FF906010E06F7040906682E084
:1025AA00FF906011E06F60048032D2D9906004E03D
:1025BA00702AA3E024F2F526E52F540744E8F583B0
:1025CA00853082740E2582F582E43583F58363A211
:1025DA000190600463A201AF26122197AE27E4FCA2
:1025EA00FDE5302528F530E52F3EF52FED352EF5A2
:1025FA002EEC352DF52DAF2CAE2BAD2AAC29AB30F8
:10260A00AA2FA92EA82DD3121A755006E5284527F8
:10261A0070099080017410F07F0022908020E52DCF
:10262A00F0A3E52EF0A3E52FF0A3E530F0908001AA
:05263A007440F0AF2622
:01263F002278
:04292B008E2B8F2C34
:10292F009068A3E0FCA3E0FDA3E0FEA3E0F5328EE8
:10293F00318D308C2FE532FFE5315407FEE42FF552
:10294F002EEE34C0F52D852E82F5837423F0052EDF
:10295F00E52E7002052D532DC7F582852D83740A40
:10296F00F0052EE52E7002052D532DC790634163A0
:10297F00A201852D83852E8263A2017F061221532A
:10298F007406252EF52EE4352DF52D852B83852CFC
:10299F008263A201852D83852E8263A201122137C6
:1029AF00908000E020E5F9E4FCFDFE9068A3E0F8DC
:1029BF00A3E0F9A3E0FAA3E02FFFEE3AFEED39FD15
:1029CF00EC38FCEF2408FFE43EFEE43DFDE43CFC64
:1029DF009068A3121A869068A3E0908040F09068E8
:1029EF00A4E0908041F09068A5E0908042F090685C
:0C29FF00A6E0908043F09080007420F06F
:012A0B0022A8
:062AE6008E2B8F2C8D2DBC
:102AEC009068A3E0FCA3E0FDA3E0FEA3E0F5338E29
:102AFC00328D318C30E533FFE5325407FEE42FF58F
:102B0C002FEE34C0F52E852F82F5837423F0052F1C
:102B1C00E52F7002052E532EC7F582852E83EBF020
:102B2C00052FE52F7002052E532EC790634163A22B
:102B3C0001852E83852F8263A2017F061221537497
:102B4C0006252FF52FE4352EF52E852B83852C822B
:102B5C0063A201852E83852F8263A201AF2D1221E2
:102B6C0053908000E020E5F97408252DF52DFFE445
:102B7C00FCFDFEE5332FF533EE3532F532ED353114
:102B8C00F531EC3530F530908040E530F0A3E5318F
:102B9C00F0A3E532F0A3E533F09080007420F0AFA1
:0D2BAC0033AE32AD31AC309068A3121A8602
:012BB90022F9
:02324C008F3FB2
:10324E009068A3E0FCA3E0FDA3E0FEA3E0F5438EAF
:10325E00428D418C40E543FFE5425407FEE42FFFCB
:10326E00EE34C09062B763A201F5838F8263A20130
:10327E00AF3F122153908000E020E5F9E4FCFDFE03
:10328E00E543253FF543EE3542F542ED3541F54137
:10329E00EC3540F540908040E540F0A3E541F0A3C9
:1032AE00E542F0A3E543F09080007420F0AF43AE0A
:0B32BE0042AD41AC409068A3121A869C
:0132C90022E2
:062A0C008E2B8F2CAB05A0
:102A12009068A3E0FCA3E0FDA3E0FEA3E0F5328E04
:102A2200318D308C2FE532FFE5315407FEE42FF56E
:102A32002EEE34C0F52D852E82F5837423F0052EFB
:102A4200E52E7002052D532DC7F582852D83EBF0FF
:102A5200052EE52E7002052D90634163A201852D9E
:102A620083852E8263A2017F061221537406252ECE
:102A7200F52EE4352DF52D532DC7E52B852E8285B8
:102A82002D83F0052EE52E7002052D532DC7F582FC
:102A9200852D83E52CF0052EE52E7002052D532D94
:102AA200C7908000E020E5F9E532240AF532E435EA
:102AB20031F531E43530F530E4352FF52F90804093
:102AC200E52FF0A3E530F0A3E531F0A3E532F09075
:102AD20080007420F0AF32AE31AD30AC2F9068A3DD
:032AE200121A863F
:012AE50022CE
:102F0000E4F526E5262401FFE433FE123676743913
:102F10002526F582E43463F583EFF00526E526C324
:102F2000943F40DFE4F526E526247FFFE433FE12DC
:102F30003676742F2526F582E43461F583EFF0743C
:102F40002F2526F582E43461F583E0FF6003B4FFAA
:102F50001D742F2526F582E43461F5837420F07406
:102F6000302526F582E43461F583E4F080090526F6
:102F7000E526C3948040B0E49061AEF0F526AF261C
:102F80007E0012367674AF2526F582E43461F5832F
:0B2F9000EFF00526E526C394FE40E3A9
:012F9B002213
:10381B00E4FDFCC3ED9FEC9E5015E4FBFA0BBB00E3
:0F382B00010ABA01F8BB90F50DBD00010C80E455
:01383A00226B
:0D38B1004390014390025390FE5390FD227E
:0D38BE005390FD5390FE4390024390012271
:0E38A2005390FD439002E5905408FF5390FDB3
:0138B00022F5
:0D38CB005390FD4390014390025390FD2265
:0738F600AE071FEE70FA227D
:02375400AD07BF
:10375600E4FC5390FDEDA804088002C333D8FC3086
:10376600E70543900180035390FE7F051238F64328
:0937760090020CBC08DC5390FD2C
:01377F002227
:1037AA00E4FF5390FD7E07439002E59030E00D74EC
:1037BA0001A806088002C333D8FC42075390FD1EB5
:0837CA00C3EE6480948050DF1F
:0137D20022D4
:10378000AB05AA071238B17FA01237541238A2AF86
:10379000021237541238A2AF031237541238A21251
:0A37A00038BE7F0A7E0012381B229B
:04367600AB07AA06EE
:10367A00C3EB94FFEA9400400DE42BF58274773A89
:10368A00F583E493FF221238B17FA012375412381F
:10369A00A2AF031237541238A21238B17FA11237DF
:0D36AA00541238A21237AA1238CB1238BEC3
:0136B70022F0
:0236F0008B2B22
:1036F200A2AF921FC2AF85A22C53A2FE8E838F82ED
:1037020005A28C838D8274091221AFE52B53A2FE90
:1037120043A2201221B153A2DF852CA2A21F92AF95
:01372200FFA7
:013723002283
:10383B00A2AF921FC2AF8C838D82EF1221AF43A236
:0C384B00201221B153A2DFA21F92AFFF98
:01385700224E
:0237D3008F263F
:1037D500A2AF921FC2AFE4F5838D8274061221AFAA
:1037E500E52643A2201221B153A2DFA21F92AF7F8B
:0137F50001D2
:0137F60022B0
:0237F7008F261B
:1037F900A2AF921FC2AFE4F5838D82740A1221AF82
:10380900E52643A2201221B153A2DFA21F92AF7F66
:0138190001AD
:01381A00228B
:10200F00A907E7FFA805EF93C3966008403B74FC50
:10201F002FFF80F00F08EF93C3966008402B74FBDF
:10202F002FFF80E00F08EF93C3966008401B74FAF0
:10203F002FFF80D00F08EF93D3966008400B74F9F1
:10204F002FFF80C01F1F1F1F1FEF54FEF80303F742
:10205F00E893FC08E893FD08E893FE08E893FF2255
:10206F0009E993C39D6008402974FB29F980F109A0
:10207F00E993C39E6008401A74FA29F980E209E9CE
:10208F0093D39F6008400B74F929F980D31919195C
:10209F001919E9C313C313FF22740093F8ECC39803
:1020AF004024701F740193F8EDC398401970147495
:0E20BF000293F8EEC398400E7009740393F874
:1020CD00EFC39840037F00227F0122EDF8E6F00870
:1020DD00A3DFFA22EDF8E0F608A3DFFA22E0A3630E
:1020ED00A201F0A363A201DFF475A20022E0A363B5
:1020FD00A201F0A363A201E0A363A201F0A363A276
:10210D0001E463A201F0A363A201DFE175A2002245
:10211D00E0A363A2016DFE936CFDEE058393FC15A8
:10212D008363A201DFEA75A200227F00E493A3631B
:10213D00A201F00F600CA3E583C2E3F58363A20156
:10214D0080EA75A20022E0A363A201F0A3E583C299
:10215D00E3F58363A201DFEE75A20022E0A363A283
:10216D0001F0A3E583C2E4D2E3F58363A201DFECC2
:10217D0075A20022E583C2E3F583E0A363A201F01B
:10218D00A363A201DFEE75A20022E583C2E4D2E3D0
:10219D00F583E0A363A201F0A363A201DFEC75A2B6
:1021AD000022F922C002C004C00612FFF0D006D0F2
:0421BD0004D0022226
:101698005452414E5A0053545245414D00525453EE
:1016A8000044454C4159004D4F4445004C494D4973
:1016B800540053495A45004C454E47544800455636
:1016C800454E504152495459004F444450415249A3
:1016D8005459004B56545F494E004B56545F4F5572
:1016E8005400574149540053544F5000003E2A2C8F
:1016F800312CCFE0F0E0ECE5F2F0FB20E0F1E8ED92
:10170800F5F0EEEDEDEEE3EE20EFEEF0F2E00A009C
:101718003E4C2C4930312C256C752CD1EAEEF0EE7C
:10172800F1F2FC20EEE1ECE5EDE02C35302C313027
:10173800302C3330302C3630302C313230302C32A3
:101748003430302C343830302C393630302C313974
:101758003230302C33383430302C35373630302C6A
:101768003131353230300A003E422C4930322C2596
:1017780062752CC2FBF1F2E0E2EBFFF2FC2052545E
:101788005320EFF0E820EFE5F0E5E4E0F7E50A00A4
:101798003E532C4930332C2562752CC7E0E4E5F024
:1017A800E6EAE020F1F2E0F0F2E020EFE5F0E5E42F
:1017B800E0F7E8282A3130ECF1290A003E422C49AA
:1017C80030342C2562752CD0E5E6E8EC20EFE5F006
:1017D800E5E4E0F7E8203720E1E8F20A003E422C91
:1017E8004930352C2562752CCFE5F0E5E4E0F7E0CB
:1017F80020F120EAEEEDF2F0EEEBFCEDFBEC20E15F
:10180800E8F2EEEC0A003E422C4930362C2562758F
:101818002CCAEEEDF2F0EEEBFCEDFBE920E1E8F28C
:10182800202D20F7E5F2EDEEF1F2FC0A003E532CF4
:101838004930372C2562752CC4EEF1F2E0E2EAE07B
:1018480020EFF0E820EFF0E8E5ECE5204E20E1E0BD
:10185800E9F220283C313236290A003E532C49301F
:10186800382C2562752CC4EEF1F2E0E2EAE020EFB4
:10187800F0E820EFE0F3E7E520EFF0E8E5ECE02022
:10188800282A3130ECF1290A003E532C4930392CF2
:101898002562752CC4EEF1F2E0E2EAE020EFF0E810
:1018A80020EFF0E8E5ECE520E1E0E9F2E02028307F
:1018B8002DEDE5F220EAEEEDF2F0EEEBFF290A005D
:1018C8003C21003C4930313D003C4930323D003C30
:1018D8004930333D003C4930343D003C4930353DCA
:1018E800003C4930363D003C4930373D003C4930EA
:1018F800383D003C4930393D000AC1F3F4E5F02099
:10190800E7E0EDFFF221000A4F55543E000A467207
:10191800616D65206572726F722120003C00FF16B0
:1019280098FF169EFF16A5FF16A9FF16AFFF16B45F
:10193800FF16BAFF16BFFF16C6FF16D1FF16DBFF4C
:0B19480016E2FF16EAFF16EFFF16F490
:10385E0052668F0000000000000000000000000013
:05386E00000000000055
:0100210022BC
:03002300022DC2E9
:0B2DC200C0E0C083C082C0D075D018F4
:102DCD00309821754701AF99D20674A1250EF58271
:102DDD00E43466F583EFF0050EE50C6005B51F02D2
:102DED00D20CC298309965300360300B07300D045A
:102DFD00D2008056E510C3950D400AC203C204D21D
:102E0D000ED20F8045AF10051074A12FF582E4345A
:102E1D0067F583E0F51330081953137F300128202F
:102E2D00D008200522631380801D30051A6313809E
:102E3D008015300112E5135213300506A2D0929B76
:0E2E4D008005A2D0B3929B851399C299D2AF93
:092E5B00D0D0D082D083D0E03247
:101BC4009068A174FFF0A374B8F0C20BE4F509C2E5
:101BD40008C201C205750840750F05F50C9068AF81
:101BE400F09068AFE075F003A42426F582E434197C
:101BF400F583E493FB740193FA740293F912195375
:101C04007003021E1BE49068B1F0A3F09068B0F07A
:101C14009068B0E0242FF582E43461F583E0FF702E
:101C240003021E129068AFE075F003A42426F58227
:101C3400E43419F583E493FB740193FA740293F981
:101C44009068B1E0F58275830012196CFEEFB50659
:101C54000F9068B27401F09068B1E004F0021E09BC
:101C64009068B2E07003021E09EE6003021E009049
:101C740068AFE0B40E004003021E12901C86F828E0
:101C84002873021CB0021CFD021D02021D07021D66
:101C940036021D6C021D6C021D6C021D9A021DA0F1
:101CA400021E12021E12021DA4021DD29068B0E090
:101CB400242FF9E43461FA7B01C0031B8B2E752FAA
:101CC40000753000E4F531D0031221C19068B312DD
:101CD4001A869068B3E0F8A3E0F9A3E0FAA3E0FB66
:101CE4007F007E8C7D0A7C001219D5121A679068D9
:101CF400A1EEF0A3EFF0021E12C209021E12D20BD3
:101D0400021E129068B0E0242FF9E43461FA7B01DA
:101D1400C0031B8B2E752F00753000E4F531D00302
:101D24001221C19068B3121A869068B6E0F50902D0
:101D34001E129068B0E0FF242FF582E43461F5832D
:101D4400E0B43702D20874302FF582E43461F583AD
:101D5400E0FFB44E04C2018002D201EF6445600387
:101D6400021E12D205021E129068B0E0242FF9E47C
:101D74003461FA7B01C0031B8B2E752F0075300074
:101D8400E4F531D0031221C19068B3121A86906829
:101D9400B6E0F5088078D201D2058072D201806E57
:101DA4009068B0E0242FF9E43461FA7B01C0031B8E
:101DB4008B2E752F00753000E4F531D0031221C14C
:101DC4009068B3121A869068B6E0F50F8040906868
:101DD400B0E0242FF9E43461FA7B01C0031B8B2E9D
:101DE400752F00753000E4F531D0031221C19068DD
:101DF400B3121A869068B6E0F50C8012E49068B2CB
:101E0400F09068B1F09068B0E004F0021C1490689F
:071E1400AFE004F0021BE542
:011E1B0022A4
:102D19007BFF7A1679F512139E9068A1E0FEA3E075
:102D2900FFC3E49FFFE49EFEAB07FA3395E0F9F891
:102D39007F007E8C7D0A7C001219D58F318E308DF3
:102D49002F8C2E7BFF7A17791812139E7BFF7A1727
:102D59007970A20BE433F52E12139E7BFF7A177953
:102D69009885092E12139E7BFF7A1779C4A208E46D
:102D790033F52E12139E7BFF7A1779E5A201E4330E
:102D8900F52E12139E7BFF7A18790EA205E433F50E
:102D99002E12139E7BFF7A18793585082E12139E01
:102DA9007BFF7A187963850F2E12139E7BFF7A18A1
:092DB9007991850C2E12139E2263
:102744007E187FC81230C1EF4E70037F01227E18BD
:102754007FCB1230C1EF4E6023123579A804A9054E
:10276400AA06AB077F007E8C7D0A7C001219D51265
:102774001A679068A1EEF0A3EFF0800A9068A17444
:10278400FFF0A374B8F07E187FD11230C1EF4E6011
:102794000C123874EF24D024FF920B8002C20B7EFB
:1027A400187FD71230C1EF4E60071235798F098038
:1027B40003E4F5097E187FDD1230C1EF4E600C1280
:1027C4003874EF24D024FF92088002C2087E187F58
:1027D400E31230C1EF4E600C123874EF24D024FFA2
:1027E40092018002C2017E187FE91230C1EF4E606F
:1027F4000C123874EF24D024FF92058002C2057EA7
:10280400187FEF1230C1EF4E60071235798F0880C0
:10281400037508407E187FF51230C1EF4E60071231
:1028240035798F0F8003750F057E187FFB1230C139
:10283400EF4E60071235798F0C8003E4F50C7F00AE
:012844002271
:10343900C203C20EC207C202C20AE4F510F50DF5B5
:103449000EF547C200D20DD20FC20CD209750BFF7F
:10345900751109122744EF6003121BC4C2ADE4F5CC
:10346900C9D2CDD2CCC2C9C2CAF5CDF5CC9068A11A
:10347900E0F5CBA3E0F5CA85CBCD85CACCE4F598B8
:1034890030010C2008095387BFD29FD29E8002D2F7
:103499009E438740C29FC2ACC298C29975B8107545
:0934A900B710D2CAD29CD2AC22A9
:0100220022BB
:102BBA00E4FF0F2407F582E43461F583E511F00F91
:102BCA0074072401F582E43461F583E4F07C667DC0
:102BDA0094FEED1DAA0470011CF5828A83E0FBAA0B
:102BEA00070F74072AF582E43461F583EBF00EBE11
:102BFA0004E07C667D98E4FEED1DAA0470011CF5D4
:102C0A00828A83E0FBAA070F74072AF582E43461FB
:102C1A00F583EBF00EBE04E07C667D9CE4FEED1DC0
:102C2A00AA0470011CF5828A83E0FBAA070F7407C5
:102C3A002AF582E43461F583EBF00EBE04E07C668B
:102C4A007DA0E4FEED1DAA0470011CF5828A83E0D2
:102C5A00FBAA070F74072AF582E43461F583EBF0C7
:042C6A000EBE04E0B6
:012C6E002243
:0A38E300C2992099FDD299D2042267
:0938ED00D2CAD29CD2ACC207225F
:1034B2008F2630030B201A5B7E197F0112292B22E3
:1034C20090637BE0F511E52624FCFFF50D7D7C750C
:1034D2008363058263A2019067A163A2011220EABD
:1034E200E4F510D203C20F300B04D200800BE509C1
:1034F2006004F54480031238E3201A157E197F0F09
:1035020012292B7E677FA1E52624FCFDE4FB122A0B
:04351200E6C20E22DD
:102F9C00E50E547FFFD394005003023032E547D343
:102FAC00950F5009EFC395085003300C79C20CC231
:102FBC0006C2AF850E12630E80530E80E4F547C235
:102FCC0002C207D2AF906478F0E512547FFFA3F0F1
:102FDC0090667CE090647AF0A3E511F0E5125480E1
:102FEC0024A1F582E43466F58363A20190647C63CA
:102FFC00A2011220EA201A29309F077E197F151290
:10300C00292B7E197F2412292BE512548024A1F53B
:10301C0082E43466AF82FEE512547FFDE4FB122A93
:09302C00E6C29F7F01227F002211
:03001E00C2AC224F
:10372400301004C210050A300008200D05C2001232
:1037340038E3E544B40106E4F5441238E330030CFD
:10374400E50AD394144008C203D20E22E4F50A22F7
:0B38D800300E05C20E7F01227F00228F
:1030410002087DE493A3F8E493A34003F68001F220
:1030510008DFF48029E493A3F85407240CC8C33390
:10306100C4540F4420C8834004F456800146F6DF5F
:10307100E4800B0102040810204080903858E47E5F
:10308100019360BCA3FF543F30E509541FFEE49354
:10309100A360010ECF54C025E060A840B8E493A31B
:1030A100FAE493A3F8E493A3C8C582C8CAC583CA46
:1030B100F0A3C8C582C8CAC583CADFE9DEE780BEFE
:013873000054
:10195300BB010689828A83E0225002E722BBFE0292
:09196300E32289828A83E49322C5
:10196C00BB010CE58229F582E5833AF583E0225030
:10197C0006E92582F8E622BBFE06E92582F8E2227A
:0D198C00E58229F582E5833AF583E4932294
:1019990075F008758200EF2FFFEE33FECD33CDCC05
:1019A90033CCC58233C5829BED9AEC99E582984088
:1019B9000CF582EE9BFEED9AFDEC99FC0FD5F0D665
:1019C900E4CEFBE4CDFAE4CCF9A88222B800C1B98F
:1019D9000059BA002DEC8BF084CFCECDFCE5F0CBCD
:1019E900F97818EF2FFFEE33FEED33FDEC33FCEB06
:1019F90033FB10D703994004EB99FB0FD8E5E4F9C1
:101A0900FA227818EF2FFFEE33FEED33FDEC33FCAD
:101A1900C933C910D7059BE99A4007EC9BFCE99AA1
:101A2900F90FD8E0E4C9FAE4CCFB2275F010EF2FE6
:101A3900FFEE33FEED33FDCC33CCC833C810D707E6
:101A49009BEC9AE899400AED9BFDEC9AFCE899F821
:0E1A59000FD5F0DAE4CDFBE4CCFAE4C8F922B4
:0E1A6700C3E49FFFE49EFEE49DFDE49CFC2290
:101A7500EB9FF5F0EA9E42F0E99D42F0E89C45F0C7
:011A8500223E
:0C1A8600ECF0A3EDF0A3EEF0A3EFF022D3
:101A9200A8828583F0D083D082121AA9121AA912C1
:101AA2001AA9121AA9E473E493A3C583C5F0C583E6
:101AB200C8C582C8F0A3C583C5F0C583C8C582C89E
:011AC2002201
:10133C00E53A242EF8E6053A22782B302602782E50
:10134C00E475F001121B24021953201FEB7F2ED2DF
:10135C001F8018EF540F2490D43440D4FF30230B4B
:10136C00EF24BFB41A0050032461FFE53B60021563
:10137C003B053EE53E7002053D30260D782BE475AD
:10138C00F001121B24EF021AC302362F7403D2266B
:10139C008003E4C226F53A8B2B8A2C892DE4F53B8D
:1013AC00F53DF53EE53B60077F2012137780F57520
:1013BC003CFFC220C21FC221C222C224C225C227A6
:1013CC00121345FF700D3026057F00121388AF3EB7
:1013DC00AE3D22B4255FC2D5C223121345FF24D0E3
:1013EC00B40A00501A75F00A783B30D50508B6FFE0
:1013FC000106C6A426F620D5047002D22280D92478
:10140C00CFB41A00EF5004C2E5D223021588D220C3
:10141C0080C6D21F80C0D22180BCD2D580BAD22443
:10142C0080B47F201213772021077401B53B004054
:10143C00F112133CFF1213770213B0D227D225807E
:10144C009512133CFB12133CFA12133CF94A4B70E5
:10145C000679597A167BFF20212EE53B602A7E0007
:10146C008E8275830012196C60060EEE653C70F06E
:10147C00C2D5EBC0E0EAC0E0E9C0E0EE1215CFD077
:10148C00E0F9D0E0FAD0E0FB121953FF60AAEBC0F0
:10149C00E0EAC0E0E9C0E0121377D0E02401F9D013
:1014AC00E03400FAD0E0FBE53C0460DCD53CD980AC
:1014BC00877BFF7A1579CBD221809C7910800279B9
:1014CC0008C225C2278008D2D5790A8004790AC2BD
:1014DC00D5E53C047002F53CE4FAFDFEFF12133C2A
:1014EC00FC7B0820201312133CFD7B10301F0A12CA
:1014FC00133CFE12133CFF7B20EC3382D592D5506B
:10150C0013C3E4301F069FFFE49EFEE42020039DDE
:10151C00FDE49CFCE4CBF8C220EC700CCFCECDCC1F
:10152C00E824F8F870F38017C3EF33FFEE33FEEDC9
:10153C0033FDEC33FCEB33FB994002FB0FD8E9EBAA
:10154C00302005F8D0E0C448B220C0E00AEC4D4E83
:10155C004F78207B0070C2EAB53C0040BCC0E01262
:10156C0015D1D0F0D0E0202004C4C0E0C4B220C01B
:10157C00F0121360D0F0D5F0EB0213B0121B8314F1
:10158C004D5314C758141E4C141A4214CB4F14D379
:0F159C004414D34914334314D95514BD4614BD18
:1015AB004514BD4716795014222D14262E14492BA1
:1015BB00142A2314472016622A13E2480000144110
:1015CB003F3F3F00790AA2D5202214302409B910DD
:1015DB00020404B9080104A2D520250250010420FD
:1015EB0021689221B53B005034C0E07F2030221996
:1015FB007F30A22172257224500F121628C221C2ED
:10160B0025C224C2277F30800F302403E9C0E012AB
:10161B001377302403D0E0F9D0E0B53BCC3024175E
:10162B007F30B9100C1213777F583023077F7880E7
:10163B0003B908031213773021057F2D0213777F2F
:10164B00202027F87F2B2025F322922180CF286E94
:10165B00756C6C2900D22012133C3020F8C2207814
:10166B003B30D50108F60213E22D504349581213B3
:10167B003C2403B405004001E490167493121368E4
:0D168B00743A121368D222753B040214C792
:1021C1008B2B8A2C892DE4F537F536F535F534F569
:1021D10032F533E52F4530452E6012EBC0E0EAC001
:1021E100E0E9C0E0AB2EAA2FA930121B34AB2B05BE
:1021F1002DE52DAA2C7002052C14F9121953F5386E
:10220100C394094007E538D3940D40E1E5386420D3
:1022110060DBE538B42D054333038016E538B42B74
:1022210005433301800C74FF252DF52D74FF352CEA
:10223100F52CE53160046410703FAB2BAA2CA92D5D
:1022410012195364306009E531702E75310A802905
:1022510090000112196CFF64786004EFB4581343C5
:1022610033017531107402252DF52DE4352CF52C33
:102271008007E5317003753108AB2B052DE52DAADB
:102281002C7002052C14F9121953F538C3946140CE
:102291000AE538D3947A50035338DF74D02538F5E2
:1022A10038C3940A400CE5389411406D74F925380F
:1022B100F538E538D39531506043330185373C8596
:1022C100363B85353A853439AF317E00E4FCFDABD0
:1022D10037AA36A935A834121AD5C8ECC8C9EDC930
:1022E100CAEECACBEFCBE4FCFDFEEB2538F537EEA9
:1022F1003AF536ED39F535EC38F534AF37AE36AD64
:1023010035FCAB3CAA3BA93AA839D3121A75500344
:1023110002227A43330402227AE53320E003E48087
:102321002DE52F4530452E601EAB2BE52D24FFF901
:10233100E52C34FFFAEBC0E0EAC0E0E9C0E0AB2EE7
:10234100AA2FA930121B34E53330E20774FFFFFED8
:10235100FDFC22E533AF37AE36AD35AC3430E103A9
:04236100021A6722D3
:101AC300BB010689828A83F0225002F722BBFE0102
:021AD300F322FC
:101AD500E88FF0A4CC8BF0A42CFCE98EF0A42CFCB0
:101AE5008AF0EDA42CFCEA8EF0A4CDA8F08BF0A42E
:101AF5002DCC3825F0FDE98FF0A42CCD35F0FCEB8D
:101B05008EF0A4FEA9F0EB8FF0A4CFC5F02ECD3951
:0F1B1500FEE43CFCEAA42DCE35F0FDE43CFC22BE
:101B2400FAE6FB0808E6F925F0F618E6CA3AF622C2
:101B3400BB011A89828A83D0F0D0E0F8D0E0F9D0D2
:101B4400E0FAD0E0FBE8C0E0C0F0021BB25016E9B6
:101B5400F8D083D082D0E0F9D0E0FAD0E0FBC082A4
:101B6400C083021BA9BBFE16E9F8D083D082D0E063
:0F1B7400F9D0E0FAD0E0FBC082C083021BBB2295
:101B8300D083D082F8E4937012740193700DA3A3F1
:101B930093F8740193F5828883E473740293686005
:061BA300EFA3A3A380DF05
:091BA900EBF608EAF608E9F62261
:091BB200EBF0A3EAF0A3E9F02234
:091BBB00EBF208EAF208E9F2225B
:00000001FF
